:020000040000FA
:040000001CEF04F0FD
:08000800E836E8363C0B010963
:10001000C212C009C216C050F80B0309C06E320EDE
:1000200019EC00F0C282C2B2FED70B6AC4500A6E4D
:100030001200036AFD0F026EFF0E00D001D00226EF
:10004000000000D000D0D8A00326D8A01200F7D717
:10005000036A056A046E076A066A100EF36E0334BB
:10006000063607360450065C0550075805E3045071
:10007000065E0550075AD88002360336F32EEFD7B6
:1000800002501200120C010C100C010C000C000CA0
:10009000000C400C840C170CD80C070C000C000C46
:1000A000010C020C030C010CAC00AC00090C020C9E
:1000B000290C000C010C010C040CA00C320C090CD6
:1000C000040C000C000C020C030C000C000C000CC7
:1000D000090C210C000C000C000C010C220C280C4B
:1000E000000C070C050C810C030C400C000C0A0CD6
:1000F000070C050C010C030C400C000C0A0C060C40
:10010000000CFF0C090C000CA10C010C090C010CDB
:10011000150C800C250C7F0C350C000C450CFF0CCD
:10012000750C080C950C080C810C020C090C020CC7
:10013000150C800C250C7F0C350C000C450CFF0CAD
:10014000750C080C950C080C910C020CC00C580195
:1001500060018801B001CC01040C030C090C040CF3
:10016000140C030C4D0C000C790C000C430C000C0F
:100170006F0C000C6D0C000C700C000C610C000C72
:100180006E0C000C790C000C140C030C4D0C000CC4
:10019000790C000C500C000C720C000C6F0C000C55
:1001A000640C000C750C000C630C000C740C000C3F
:1001B0000E0C030C310C000C320C000C330C000C38
:1001C000340C000C350C000C360C000C030C030C2A
:1001D000000C04011E51600B00083EE1050E1F6378
:1001E00003D0040E1A6F36D0060E1F6301D035D02F
:1001F000080E1F6309D01B0E126F040E136F010E41
:10020000186F196B1D9326D0090E1F6301D067D09C
:10021000000E1F6301D07BD0010E1F6301D09CD064
:10022000030E1F6301D098D00A0E1F630BD01C0E63
:10023000126F040E136F22511227010E186F196BE3
:100240001D9308D00B0E1F63120024EE1CF02251E8
:1002500020C4DBFF010E176F1200800E1E63120018
:10026000010E21630ED0840E126F136B12C4F6FFC1
:1002700013C4F7FFF86A0800F5CF18F4196B1D8353
:10028000E9D7020E216310D0AC0E126F136BB00EC3
:10029000F66EF76AF86A0900F5CF18F4090008004D
:1002A000F5CF19F41D83D6D7030E21631200F86A27
:1002B000F76A20454E0FF66E010EF7220900F5CFC2
:1002C00012F40800F5CF13F412C4F6FF13C4F7FFBD
:1002D000F86A0800F5CF18F4196B1D83BBD7010E1F
:1002E000176F2FEE71F00F0EDE6AE82EFDD724EEA9
:1002F0001CF0010EDE6AE82EFDD720511B6F03E1D2
:10030000050E1A6F1200060E1A6FFFD912005E6BEF
:100310005F6B1E511F0B000803E11DB15E830ED001
:100320001E511F0B010801E109D01E511F0B0208CD
:1003300007E134D8DF50040B01E05E81010E176F36
:10034000010E176312005E0E126F040E136F020E81
:10035000186F196B1D931200010E206309D01E51F6
:100360001F0B000805E11D81030E1F631D9172D74D
:10037000000E206312001E511F0B0208FBE12251E8
:100380000F0BF8E00BD8030E1F6303D0840EDF6E53
:1003900061D7000E22AF880EDF6E5CD724EE00F02E
:1003A00022452235E846E846D9261200000E6C6246
:1003B00005D000513C0B340805E00FD0040E6C62F0
:1003C000120014D0000E166F176B186B196B01DF3B
:1003D000000E176378D040D976D0020E1663AED0E7
:1003E00056D8C80E00BD880E006F1200040E1A63A6
:1003F00006D020516E6E050ED8B4030E1A6F010E92
:1004000016639CD005D8C80E04BD880E046F120078
:100410001851106F1951116F000804E306E11851CB
:10042000400803E2400E106F116B1051056F185F0A
:100430001151195B0451FC0B1111046F24EE5EF095
:10044000115102E1105122E01DA312D012C4F6FF97
:1004500013C4F7FFF86A0900F5CFDEFF09001007A3
:10046000FAE11107F8E2F6CF12F4F7CF13F4120015
:1004700012C4E1FF13C4E2FFE6CFDEFF1007FCE188
:100480001107FAE2E1CF12F4E2CF13F412000151A6
:10049000106F18270051030B116F192314EE5EF033
:1004A00014C4D9FF15C4DAFF115102E110510AE05A
:1004B000E6CFDEFF1007FCE11107FAE2D9CF14F412
:1004C000DACF15F41200000E17630AD0400E016F48
:1004D0001E0E026F040E036F840E006F046F2CD08B
:1004E0001EAF1DD01951255D04E307E11851245DAD
:1004F00004E224C418F425C419F48ADF010E166F2F
:10050000400E016F1E0E026F040E036F800E006F0F
:100510005E0E066F040E076FC80E046F0DD0020E3C
:10052000166F056BC80E046F400E016F5E0E026FF2
:10053000040E036FC80E006F6D981200000E166F48
:10054000400E016F1E0E026F040E036F880E006FC7
:10055000000E046F12000401140E6F6E1A6B1D6BF7
:100560001B6BD3D8120004016DA60CD8010E1A63C0
:1005700012006DBA1200686A696A69806988020EA1
:100580001A6F12006D6A696A6D86010E1A6F120089
:100590006D6A696A1A6B12000401000E1A5D23E08D
:1005A00068A402D069B424D86DB2120068A002D049
:1005B00069B038D868A802D069B816D868AC02D03B
:1005C00069BC27D868AA02D069BA25D868A202D027
:1005D00069B226D8030E1A5D06E368A604D069A6A0
:1005E00002D0E4DE68961200698468986D82120079
:1005F0006D926994689412001DA11200F9DF6D8458
:10060000100EF46EF36AF32EFED7F42EFCD76D9421
:100610001200689C120070B091DF7090689A12000E
:10062000689212006A6A686A9F0E6B6E7B0E696E32
:100630006E6A2FEE71F00F0EDE6AE82EFDD7160EF1
:10064000706E68B6689668B6FDD76D9877DF1D91B5
:100650001B6B030E1A6F120004011E511F0B0108C1
:1006600002E1000E22631200060E1F6324D0210E49
:1006700021630ED0D00E126F136B12C4F6FF13C499
:10068000F7FFF86A0800F5CF18F4196B1D833AD00C
:10069000220E216310D0FE0E126F136BDE0EF66E6B
:1006A000F76AF86A0900F5CF18F409000800F5CFD9
:1006B00019F41D8327D01E51600B2008D4E1020ECF
:1006C0001F6309D09E0E126F040E136F010E186F78
:1006D000196B1D9317D00A0E1F6303D021C49EF41B
:1006E00011D0030E1F6309D09F0E126F040E136FFB
:1006F000010E186F196B1D9305D00B0E1F631200AE
:1007000020C49FF4020E176F1200010EE96E16EE60
:1007100000F0400EE66E2FEE70F0E950D9261C0E68
:10072000DF12E944E846E84604EE00F0E926020E4E
:10073000E1CFEBFF030EE2CFEBFFE550E92AE7CF75
:10074000EDFF880EEF6E010EE96E15EE10F0400E13
:10075000E66E2FEE70F0E950D9261A0EDF12E9444A
:10076000E846E84604EE04F0E926020EE1CFEBFF8E
:10077000030EE2CFEBFF400EEF6E1200066E53D871
:100780000044E846E84604EE00F0E926E86AD8802E
:10079000EFBE1200020EEBCFD9FF030EEBCFDAFF54
:1007A000EC500660066EFF0EDB50ED6E065004E066
:1007B000DECFE6FFE82EFCD7400EEF16EF7C880E6A
:1007C000EF120650D8901200066E05EE11F0E6CF3B
:1007D000EEFFE82EFCD701D0066E25D80AD8D8B097
:1007E00007D019D8400EEF16EF7C880EEF12D89084
:1007F00012000044E846E84604EE04F0E926E86A00
:10080000D880EFBE1200020EEBCFD9FF030EEBCF64
:10081000DAFFD8901200FF0EDB500660066EE92A60
:100820000650ED6E1200E0CF03F09DDEB5DE1AC477
:1008300002F003C0E0FF1200F86A8DDE0001AB6A2F
:10084000C190C192C184C1960F6A0E6A7DEC04F01A
:10085000000E04EC00F00C6E0CC012F00CC002F0A4
:100860000A0E28EC00F0016E01C013F0036A0CC000
:1008700002F0056A0A0E046E2BEC00F006C001F0CF
:1008800001C014F00A0E04EC00F00D6E0DC015F05E
:100890000DC002F00A0E28EC00F0016E01C016F047
:1008A000036A0DC002F0056A0A0E046E2BEC00F01C
:1008B00006C001F001C017F0010E006E10EE11F03D
:1008C000080E82DF010E006E10EE11F0080E56DFEA
:1008D000D8B0BED7BDD7010E006E10EE11F0080ED5
:1008E0004DDFD8B0F8D71200010E006E10EE11F0F7
:1008F000080E6ADFD8B0F8D7120095DF060E025C4A
:06090000D8A4FBD7120091
:020000040030CA
:08000000E4FEFFEEFFFD9BFF93
:00000001FF
